:1000000009C0222728BB27BB089521E0E20F20E08A
:10001000F21F0895F894479AE0EEF0E0C895302C6E
:10002000F4DFC895202CF1DFC895502CEEDFC89581
:10003000402CEBDFC895702CE8DFC895602CE5DF1D
:10004000C895902CE2DFC895802CC8EED0E0EC2F4C
:10005000FD2F5527662703E030E841E05395501304
:100060000FC0552703E028E0C20F20E0D21F6395A0
:1000700026E1621305C06627C8EED0E0EC2FFD2F05
:100080003215430538F0C895C0DF08BAC89507BADD
:10009000B8DFBBDF3415450538F0C895B6DF08BAC0
:1000A000C89507BAAEDFB1DF3615470538F0C895F9
:1000B000ACDF08BAC89507BAA4DFA7DF3815490531
:1000C00030F0C895A2DF08BAC89507BA9ADFEC2FBE
:1000D000FD2F3150404022273217420789F6BCCF0E
:1000E00000010100014001700212101201111011F3
:1000F0001014021210120111041410140212101222
:10010000010504141014021204050105041410144E
:10011000010304050105041402030103040501059C
:100120000406020301030405020604060203010398
:100130000406020600000203020304060206000091
:100140000103020304060206040501030203040678
:10015000010504050103020304140105040501035C
:1001600010140414010504050212101404140105EE
:1001700010120212101404140111101202121014A1
:1001800010110111101202120111101100001012B1
:08019000101201111011000012
:00000001FF
